:1000000018308A00002800000A108A100A1182079E
:1000100028340C34013406340A108A100A1182077D
:100020000E341134113415340E340E340E340434BD
:1000300014340A3400340E340B340E341A340E34B3
:1000400000340834143408340334043404340334DE
:10005000043414340434143404340E340E340434AC
:1000600000340A34153400340A34153400340034B2
:1000700000340034003411340A340E3400340034B7
:1000800000340E341534173411340E340034003477
:100090000834023408340034043400341F3400348B
:1000A00000340034003400340034003400340034B0
:1000B0000A108A100A115F3E03188A0A820000346F
:1000C0005E34BC34E23461343F34DD348334C234D2
:1000D0009C347E342034A334FD341F3441349D34A9
:1000E000C33421347F34FC34A23440341E345F34B2
:1000F0000134E334BD343E3460348234DC342334A0
:100100007D349F34C13442341C34FE34A034E13495
:10011000BF345D3403348034DE343C346234BE3466
:10012000E03402345C34DF34813463343D347C3475
:100130002234C0349E341D344334A134FF34463459
:100140001834FA34A434273479349B34C5348434D5
:10015000DA3438346634E534BB3459340734DB34AC
:10016000853467343934BA34E434063458341934B5
:100170004734A534FB3478342634C4349A34653497
:100180003B34D934873404345A34B834E634A73491
:10019000F9341B344534C63498347A342434F83472
:1001A000A63444341A349934C73425347B343A3471
:1001B00064348634D8345B340534E734B9348C3451
:1001C000D23430346E34ED34B33451340F344E34D1
:1001D0001034F234AC342F3471349334CD341134C0
:1001E0004F34AD34F33470342E34CC349234D334B1
:1001F0008D346F343134B234EC340E345034AF3487
:10020000F13413344D34CE34903472342C346D3494
:100210003334D1348F340C345234B034EE3432347D
:100220006C348E34D03453340D34EF34B134F03474
:10023000AE344C3412349134CF342D347334CA3448
:10024000943476342834AB34F534173449340834D4
:100250005634B434EA3469343734D5348B345734B3
:100260000934EB34B534363468348A34D4349534B4
:10027000CB3429347734F434AA3448341634E9348E
:10028000B73455340B348834D63434346A342B3490
:1002900075349734C9344A341434F634A834743479
:1002A0002A34C834963415344B34A934F734B63470
:1002B000E8340A345434D73489346B34353420105C
:1002C0002010201000003C00EF3500013E000C0023
:1002D000553A723DF9367535A012751000000C00C4
:1002E000C737643D6937611025183232201000008D
:1002F0000C00CD34EE3AF430A01230196410200016
:100300000C00D332EB3A6E32A01230196410200088
:100310008C27F03AF331A036653775000C000C2AB3
:10032000E536F032F230F43AF23000010C008C2B5A
:100330006C17EF39F734653AEC32EE3461008C2AF1
:10034000733AE13BE937EE37A0123019641D2518E6
:10035000323200010C008C2B7936AE37F33BE93298
:1003600074366537E93000018C2A733AE13BE9378E
:10037000EE37A0123019641D2518323200010C002E
:100380000C276138EF3BE9327439FA30EE346500FE
:100390008C2AF23A6334EF36E932EE346505E337FE
:1003A000A01230196410E81725183232A0366937C8
:1003B00000010C008C256139ED346537E93200010C
:1003C0008C2AF23A6334EF36E932EE346505E337CE
:1003D000A01230196410E81725183232A039000134
:1003E0000C000C2DE533613900018C2A733AE13B96
:1003F000E937EE37A0123019641D2518323200019A
:100400000C000C2AE539F43A6A000C3AE539741DFF
:1004100000010C000C27EF3BE522EE32F233E9320B
:10042000AE37F2330A3B33000C2A6539ED37ED3233
:1004300074390A3DE134EE39F430EC37F730EE3CF4
:100440002E000C286F32EC30633D0A3A6539ED37E7
:10045000ED3274392100200020002000200020000F
:100460007C308400831300080319432A0630F80007
:10047000F701F70B392AF80B382A7B30F700F70B16
:100480003F2A800B362A08007B18482A0812492A7E
:10049000081683160812FB18512A83128712532A52
:1004A000831683128716A0122008831687007B19F3
:1004B0005D2A831207125F2A831683120716201201
:1004C000200883168700FB19692A831288116B2A7A
:1004D00083168312881583168811000088128312F0
:1004E00088160230F700F70B732A762A000083166D
:1004F0008812831288120800FC0183168812831266
:1005000088160000831608167C108312081A7C14C3
:10051000A016200883168700FC108312871AFC148B
:1005200020162008831687007C118312071A7C1579
:1005300083168815FC1183128819FC1583168812FE
:10054000831288127C08F80008008316881383122F
:100550008813831608138312081700007C2278087A
:10056000FB007C227808F6007B0EF700F030F705E0
:1005700077087604F8007808F600F61BA92AF40834
:100580000319C72A8316881383128817CB2A831668
:10059000881383128813000083160813831208132C
:1005A00000008316881283128812750EF6000F3031
:1005B000F6057608FB00442275080F39F600FB00AB
:1005C00044220800831688138312881383160813A5
:1005D0008312081383168812831288120F30FC00CE
:1005E0003022DE015E08023C031CFE2A0330FB00C1
:1005F00044220530FC003022DE0AF22A0230FB00E1
:100600004422DE015E08033C031C0F2B5E0804201D
:10061000DF00F4015F08F500A522DE0A022B8A152F
:100620000A164328F4014030F500A522DE015E08D9
:100630003F3C031C282B5E080C20DF000130F40037
:100640005F08F500A5220230FC003022DE0A172BDD
:100650008A150A164828710B2E2B312B4030F200D8
:10066000322BF20101307002F20772088038F30079
:10067000F4017308F500A52208006F080C3A03196D
:10068000482B063A0319502B023A0319562B5B2BC1
:10069000F4010130F500A5220230FC003022602B6D
:1006A0000130F0000230F1002B23602BF4011030F8
:1006B000F500A522602B0130F4006F08F500A5229B
:1006C00008000B08E2008B13831603178C170C1419
:1006D0000000000083120313E21B8B1703170C08A2
:1006E0007F390319B52B0313E20003170D08031319
:1006F000E30003170F080313E4006208EF003D2333
:10070000630803178D000313640803178F00031396
:100710000B08E5008B13831603178C170C140000CD
:10072000000083120313E51B8B1703170C0D0E0D2E
:100730007F390319B52B0313E20003170D080313C8
:10074000E30003170F080313E4006208EF003D23E2
:10075000630803178D000313640803178F008D0AC5
:1007600003198F0A0313612B0317031308000330C7
:10077000FE02031CC52B7E3084008313000803197E
:10078000C52BC32BC32B800BC22B080083168611ED
:10079000831286110330FD00C330FE00B723FD0B2A
:1007A000CC2B831686158830F700F70BD52B00006D
:1007B0008615FC0183128619FC0A0230FD00D33035
:1007C000FE00B723FD0BDF2B7C08F8000800831622
:1007D0008611831286118316210BF52B1630F70034
:1007E000F70BF02BF32B00008615F130F700F70B19
:1007F000F72B0000861583120800FE017E08073CD7
:10080000031C1A2C7D088316A0007E08F80003192B
:100810000D2C0310A00CF80B092C0130A0052008AA
:10082000A1008312E7231830F700F70B152C182CC2
:10083000FE0AFE2BCF30F700F70B1C2C1F2C0000FC
:10084000080083168611831286111630F700F70B05
:10085000272C2A2C0000831686151630F700F70B7C
:100860002F2C322C0000861500308312861901309F
:10087000F80008000130E000E101E200E301E401DA
:10088000E601C401C62367107818671467184A2C5C
:100890002A1C4E2CA9010030F800CB2CF030FD00B2
:1008A000FD23E3012124780B572C0230E300FA30BA
:1008B000FE00B7232124780B5E2C63146308033CED
:1008C000031D642CBB2CB72CE30803196B2C0310FD
:1008D000630CE500892C2908600203187C2C213068
:1008E00061078400831300086205031D792C003022
:1008F0007A2C0130E500842C290860020319822C2F
:100900000030832C0130E500E508031D892C6008C8
:10091000E400650B932C21306107840083130008E9
:10092000620480009B2C21306107840083136208DD
:10093000FF3A0005800065088316A1008312E723B3
:10094000E00A0310E20DE208031DB72C2130610715
:10095000840083130008E8006808E9004408690679
:100960005820F800C4004408F800E10AE20A6108CF
:10097000073C0318512C6008403C031CC12CA90102
:10098000C92C6408A9002A10A90803192A140130E7
:10099000E6006608F8000800DF01C623F808031D1A
:1009A000002DA9012A103A247808F8080319002D0F
:1009B000C301C30ADF0ADE015E08073C031CFC2CEE
:1009C000430DF700F70DF70DF830F70577085E07D0
:1009D0002B3EF800FA010318FA0A21305E07840062
:1009E00083130008E2007808840083137A188317C1
:1009F00062088000DE0ADC2C3A24F808031DD92C9A
:100A00005F08F8008A150A166328E2010130E10048
:100A10000830F8001F08C73978049F000F2D102DEB
:100A200000001F151F19122D83161E088312E100E6
:100A30001E08E2000130FC0030226208E400610878
:100A4000E3006408013C0318552DFF3A031D2C2DCB
:100A50006308583C0318552D6408033C031C552DAE
:100A6000031D362D6308B53C031C552D4508033C7A
:100A7000031D422D0130C5070130FC003022023039
:100A8000F8007A2D4508033C031C552D0130C5079D
:100A90000230E500FA30FC003022E50B4A2D01302F
:100AA000FC0030220030F8007A2D6408023C031C60
:100AB000662D031D5F2D6308573C031C662DC50181
:100AC0000130FC0030220330F8007A2D6408023C2B
:100AD0000318782DFF3A031D712D6308B63C0318E7
:100AE000782DC5010130FC0030220130F8007A2D4C
:100AF0000030F800780808008316881083128814E4
:100B00005E08FC003022831688108312881005309E
:100B1000FC00302208000130F0000230F1002B23ED
:100B2000633003178D0001308F00031361230830F9
:100B3000F0000230F1002B23643003178D000130E8
:100B40008F00031361231030F0000230F1002B23DB
:100B5000663003178D0001308F00031361230800F6
:100B60000B08E2008B13831603178C170C1400007C
:100B7000000083120313E21B8B170318E72D0317E2
:100B80000C087F390313E20003170D080313E30079
:100B900003170F080313E4006208EF003D23630806
:100BA00003178D000313640803178F0003130B084A
:100BB000E5008B13831603178C170C14000000003C
:100BC00083120313E51B8B17E10BE72D062E03178A
:100BD0000C0D0E0D7F390313E20003170D080313EC
:100BE000E30003170F080313E4006208EF003D233E
:100BF000630803178D000313640803178F008D0A21
:100C000003198F0A03100313E10BB02D08006808C5
:100C1000F801670203180F2E6708F7001B2EF70173
:100C20000830E900E70DF70D680877020318F700B0
:100C3000F80DE90B122E08002030621E3030E30060
:100C40006108F700E11F2C2EF709F70A7708E10089
:100C50002D30E300E21762146108E7006430E80019
:100C600007267708E10030307807E4006108E700E4
:100C70000A30E800072630307707E6003030780782
:100C8000E5006308F7003030640203194B2EE214CC
:100C9000E21B62155F2E62195F2E6308E400E21802
:100CA000562E303065020319592E6214E21BE214ED
:100CB0005F2E031D6214031D5F2E6408E500621998
:100CC000662EE218692E62186C2E6F2E6308EF00F4
:100CD0003D236408EF003D236508EF003D236608CF
:100CE000EF003D23080060146F3003178D000130C2
:100CF0008F00031361238B250430E100C830FC0012
:100D00003022E10B7E2E601CC22E0430E100C83080
:100D1000FC003022E10B872E0230F0000130F100A0
:100D20002B23703003178D0001308F000310083023
:100D30000313E100B0255F08E1000130E2001C264A
:100D40002030EF003D232030EF003D2305257808BB
:100D5000033A0319B22E023A0319B92E033A0319C2
:100D6000C02EC12E0130DF025F0FB82E1830DF0019
:100D7000C12E0130DF075F08183C031CDF01C12EC4
:100D80006010832E5F08F8000800601478300317A5
:100D90008D0001308F00031361238B250430E100A7
:100DA000C830FC003022E10BD02E601C142F043020
:100DB000E100C830FC003022E10BD92E0230F000F7
:100DC0000130F1002B23793003178D0001308F00A3
:100DD000031007300313E100B0255F08E100013084
:100DE000E2001C262030EF003D232030EF003D23A1
:100DF00005257808033A0319042F023A03190B2F2B
:100E0000033A0319122F132F0130DF025F0F0A2F4D
:100E10003B30DF00132F0130DF075F083B3C031C32
:100E2000DF01132F6010D52E5F08F80008005E0860
:100E3000E7000A30E8000726780EDF00F030DF0513
:100E40005E08E7000A30E800072677085F07F80029
:100E500008000830F8000430F700F70B2D2F86103B
:100E6000831686100330F700F70B342F8312E30D3F
:100E70000610031C3E2F8316061483120318432FFB
:100E8000831606108312831686148312861C462F3F
:100E9000F80B2B2F0430F700F70B4C2F861083161E
:100EA0008610000006140330F700F70B552F0330AF
:100EB000F700F70B592F86148312861C5D2FF8015B
:100EC0000330F700F70B622F06187814861083168C
:100ED00086108312061083160610831208008316EC
:100EE00006140430F700F70B732F86140330F70055
:100EF000F70B782F83120610831606100430F700C4
:100F0000F70B802F8312861083168610D030831241
:100F1000E30029275F08E30029276008E300292769
:100F200083160610000086148312861C952F043049
:100F3000F700F70B992F9C2F00008316061404303E
:100F4000F700F70BA12F06140430F700F70BA62FBC
:100F500086140330F700F70BAB2F831206108316AD
:100F600006100430F700F70BB32F83128610831698
:100F70008610D0308312E300292778086110781892
:100F80006114D030E2006118C92F6208043C031CD0
:100F9000EC2F831606140430F700F70BCD2F8614C0
:100FA0000330F700F70BD22F8312861CD52F0610C3
:100FB000831606100430F700F70BDC2F831286101F
:100FC00083168610D0308312E30029277808611039
:100FD00078186114E20AC32F08005F0EF7000F3083
:100FE000F7057708E100E2000A30E3008A15BD2624
:100FF0008A117808E0005F080F396007F8000800E0
:10100000460B0E284708063C031C0E28AA180E287B
:10101000C70A0A30DE008A117C258A154608033C7F
:10102000031D1E284708003C03181E28AA181E2866
:10103000C7030A30DE008A117C258A154608023C67
:10104000031D2528C708031DAA144708F83E0318E6
:10105000102E083E132E883003178D0001308F00AC
:101060008A11031361238A158A118B258A1504308E
:10107000DE00FA30FC008A1130228A15DE0B392896
:10108000AA10C7018E3003178D0001308F008A111E
:10109000031361238A15102E8F3003178D00013042
:1010A0008F008A11031361238A158A118B258A15F3
:1010B000AA1C2B295E1403178D0183168C130C14A4
:1010C00083120C080313DF005F0F68281930DF005C
:1010D000673003178D0001308F008A1103136123DD
:1010E0008A158A118B258A150430E000C830FC006F
:1010F0008A1130228A15E00B76285E1C16290430EE
:10110000E000C830FC008A1130228A15E00B8128EB
:101110000230F0000130F1008A112B238A1568306B
:1011200003178D0001308F00031009300313E10015
:101130008A11B0258A155F08E0001B30E1006008C5
:10114000E7006430E8008A1107268A157708E00076
:1011500078083030031DB328E11CBC28E119BC28F5
:10116000611A2030B628E11161126114F80778087D
:10117000EF008A113D238A156008E7000A30E80075
:101180008A1107268A157708E00078083030031D99
:10119000CF28E119D528611CD528611A2030F8071D
:1011A0007808EF008A113D238A153030E007600887
:1011B000EF008A113D238A152030EF008A113D236C
:1011C0008A150130F4000230F5008A11A5228A1533
:1011D0008A1105258A157808033A0319F628023A78
:1011E0000319F928033A0319FC2815290130DF02F5
:1011F00015290130DF0715290B08F7008B1303179A
:101200008D0103135F0803178C0083168C130C15D4
:1012100055308D00AA308D008C148C180D290C11BE
:101220007708831203138B045E107D280A30DE00DA
:101230008A117C258A150A30DE008A117C258A15E0
:10124000AA10C701963003178D0001308F008A1154
:10125000031361238A15102E973003178D00013078
:101260008F008A11031361238A158A118B258A1531
:10127000AA1CDF29013003178D0083168C130C1470
:1012800083120C080313DE005E08DF008A11732648
:101290008A157808DE000B08F7008B13013003175E
:1012A0008D0003135E0803178C0083168C130C1536
:1012B00055308D00AA308D008C148C185D290C11CE
:1012C0007708831203138B04023003178D008316F3
:1012D0008C130C1483120C080313DE005E08DF006D
:1012E0008A11C5268A157808DE000B08F7008B13D3
:1012F000023003178D0003135E0803178C0083165A
:101300008C130C1555308D00AA308D008C148C1860
:1013100087290C117708831203138B0401300317FC
:101320008D0083168C130C1483120C080313DE003B
:10133000023003178D0083168C130C1483120C08D3
:101340000313DF009F3003178D0001308F0003105F
:101350000B300313E1008A11B0258A155E08E10005
:101360000130E2008A111C268A153A30EF008A11FA
:101370003D238A155F08E1000130E2008A111C2636
:101380008A150830DE00FA30FC008A1130228A15F6
:10139000DE0BC3290A30DE008A117C258A150A304B
:1013A000DE008A117C258A15AA10C701AA3003170E
:1013B0008D0001308F008A11031361238A15102ECE
:1013C000AB3003178D0001308F008A1103136123A6
:1013D0008A158A118B258A15AA1C932A03300317B4
:1013E0008D0083168C130C1483120C080313DE007B
:1013F0005E08DF008A1173268A157808DE000B0864
:10140000F7008B13033003178D0003135E080317D7
:101410008C0083168C130C1555308D00AA308D006E
:101420008C148C18112A0C117708831203138B0467
:10143000043003178D0083168C130C1483120C08D0
:101440000313DE005E08DF008A11C5268A157808BE
:10145000DE000B08F7008B13043003178D00031315
:101460005E0803178C0083168C130C1555308D0005
:10147000AA308D008C148C183B2A0C11770883122B
:1014800003138B04033003178D0083168C130C1485
:1014900083120C080313DE00043003178D0083163B
:1014A0008C130C1483120C080313DF00B4300317E1
:1014B0008D0001308F0003100B300313E1008A11FF
:1014C000B0258A155E08E1000130E2008A111C2671
:1014D0008A153A30EF008A113D238A155F08E10032
:1014E0000130E2008A111C268A150830DE00FA302D
:1014F000FC008A1130228A15DE0B772A0A30DE00C2
:101500008A117C258A150A30DE008A117C258A150D
:10151000AA10C701BF3003178D0001308F008A1158
:10152000031361238A15102EC03003178D0001307C
:101530008F008A11031361238A158A118B258A155E
:10154000AA1C5E2BCB01073003178D0083168C136A
:101550000C1483120C080313DE005E08DF008A11EE
:1015600073268A157808DE000B08F7008B13073006
:1015700003178D0003135E0803178C0083168C136A
:101580000C1555308D00AA308D008C148C18C62A8D
:101590000C117708831203138B04083003178D0096
:1015A00083168C130C1483120C080313DE005E08E0
:1015B000DF008A11C5268A157808DE000B08F700BF
:1015C0008B13083003178D0003135E0803178C007C
:1015D00083168C130C1555308D00AA308D008C1499
:1015E0008C18F02A0C117708831203138B04073030
:1015F00003178D0083168C130C1483120C0803132D
:10160000DE00083003178D0083168C130C14831230
:101610000C080313DF00C83003178D0001308F0062
:10162000031011300313E1008A11B0258A155E08FA
:10163000E1000130E2008A111C268A152030EF00FB
:101640008A113D238A156830EF008A113D238A15DF
:101650002F30EF008A113D238A155F08E100013029
:10166000E2008A111C268A15D63003178D0001303E
:101670008F00031004300313E1008A11B0258A158E
:101680000830DE00FA30FC008A1130228A15DE0BA9
:10169000422B0A30DE008A117C258A150A30DE00D2
:1016A0008A117C258A15AA10C701D93003178D002D
:1016B00001308F008A11031361238A15102EDA304E
:1016C00003178D0001308F008A11031361238A15DF
:1016D0008A118B258A15AA1C892CCC010530031789
:1016E0008D0083168C130C1483120C080313DE0078
:1016F0005E08DF008A1173268A157808DE000B0861
:10170000F7008B13053003178D0003135E080317D2
:101710008C0083168C130C1555308D00AA308D006B
:101720008C148C18912B0C117708831203138B04E3
:10173000063003178D0083168C130C1483120C08CB
:101740000313DE005E08DF006014803003178D0095
:1017500001308F008A11031361238A158A118B25AA
:101760008A150430E100C830FC008A1130228A1545
:10177000E10BB32B601C072C0430E100C830FC00E7
:101780008A1130228A15E10BBE2B0230F0000130A5
:10179000F1008A112B238A15813003178D00013047
:1017A0008F00031007300313E1008A11B0258A155A
:1017B0005F08E1000130E2008A111C268A15203002
:1017C000EF008A113D238A152030EF008A113D2356
:1017D0008A158A1105258A157808033A0319F72B0B
:1017E000023A0319FE2B033A0319052C062C01308B
:1017F000DF025F0FFD2B3B30DF00062C0130DF07DF
:101800005F083B3C031CDF01062C6010BA2B5F080D
:10181000F8007808DE000B08F7008B13063003177A
:101820008D0003135E0803178C0083168C130C15B0
:1018300055308D00AA308D008C148C181D2C0C1185
:101840007708831203138B04053003178D0083166A
:101850008C130C1483120C080313DE0006300317DC
:101860008D0083168C130C1483120C080313DF00F5
:10187000E03003178D0001308F0003101130031387
:10188000E1008A11B0258A155E08E1000130E2000E
:101890008A111C268A152030EF008A113D238A15F3
:1018A0006830EF008A113D238A152F30EF008A112E
:1018B0003D238A155F08E1000130E2008A111C26F1
:1018C0008A152030EF008A113D238A157330EF000E
:1018D0008A113D238A150830DE00FA30FC008A1197
:1018E00030228A15DE0B6D2C0A30DE008A117C2531
:1018F0008A150A30DE008A117C258A15AA10C701D4
:10190000F03003178D0001308F008A11031361231B
:101910008A15102EF13003178D0001308F008A11C7
:10192000031361238A158A118B258A15AA1C342D6D
:101930004A08DF008A1173268A157808CA00490808
:10194000DF008A11C5268A157808C900F53003170B
:101950008D0001308F0003100B300313E1008A115A
:10196000B0258A154A08E1000130E2008A111C26E0
:101970008A153A30EF008A113D238A154908E100A3
:101980000130E2008A111C268A150130DE008A111E
:1019900017278A157808DE000430DF007808E00099
:1019A0008A116F278A150130DE008A1117278A15E0
:1019B0007808DE000530DF007808E0008A116F2724
:1019C0008A15DE018A1117278A157808DE0006308D
:1019D000DF007808E0008A116F278A154A08DE00C8
:1019E0008A1117278A157808DE000230DF00780890
:1019F000E0008A116F278A154908DE008A1117272F
:101A00008A157808DE000130DF007808E0008A11CE
:101A10006F278A15DE018A1117278A157808DE00DC
:101A2000DF017808E0008A116F278A150C30DE008C
:101A3000FA30FC008A1130228A15DE0B182D0A308C
:101A4000DE008A117C258A150A30DE008A117C2589
:101A50008A15AA10C701003003178D0002308F00CD
:101A60008A11031361238A15102E013003178D008C
:101A700002308F008A11031361238A158A118B2586
:101A80008A15AA1C102E0A30DE008A117C258A15C0
:101A90000A30DE008A117C258A15053003178D0077
:101AA00002308F008A11031361238A150630F0007B
:101AB0000130F1008A112B238A150130F400F50161
:101AC0008A11A5228A15A010200883168700831288
:101AD00087140830DE00FA30FC008A1130228A15A3
:101AE000DE0B6B2DA0102008831687008312871051
:101AF0000C30DE00FA30FC008A1130228A15DE0B31
:101B00007A2D0630F0000130F1008A112B238A155E
:101B10000130F400F5008A11A5228A15A0102008D2
:101B200083168700831287140830DE00FA30FC0029
:101B30008A1130228A15DE0B962DA01020088316FC
:101B40008700831287100C30DE00FA30FC008A1107
:101B500030228A15DE0BA52D0630F0000130F10091
:101B60008A112B238A150130F4000530F5008A1103
:101B7000A5228A15A01120088316870083128715D5
:101B80000830DE00FA30FC008A1130228A15DE0BA4
:101B9000C22DA011200883168700831287110C30F4
:101BA000DE00FA30FC008A1130228A15DE0BD12DBE
:101BB0000630F0000130F1008A112B238A15013024
:101BC000F4000730F5008A11A5228A158316081043
:101BD000831208140830DE00FA30FC008A1130222B
:101BE0008A15DE0BEC2D83160810831208100C30BA
:101BF000DE00FA30FC008A1130228A15DE0BF92D46
:101C0000AA10C7010A30DE008A117C258A15093026
:101C100003178D0002308F008A11031361238A1588
:101C20008A150A16A3280A108A140A1582072B2877
:101C30004C282C29E029942A5F2B8A2C352D8316D9
:101C400006140430F700F70B232E86140330F70038
:101C5000F70B282E8312861C2B2E061083160610D7
:101C60000430F700F70B322E83128610831686108D
:101C7000D0308312E3008A1129278A155E08E30019
:101C80008A1129278A15831606140430F700F70BEA
:101C9000472E86140330F700F70B4C2E8312861C58
:101CA0004F2E0610831606100430F700F70B562E41
:101CB0008312861083168610D1308312E3008A11B6
:101CC00029278A15F7010830E1007708E20083161A
:101CD00006140330F700F70B6B2E86148312861C54
:101CE0006F2E06180314061C0310F80D0430F700BD
:101CF000F70B782E8316861083128610E10B672E61
:101D0000831606140330F700F70B842E8312061097
:101D1000620803198E2E83160610831200008316A4
:101D200086148312861C922E0430F700F70B962E31
:101D30008610831686100330F700F70B9D2E831252
:101D400006108316061078088312DF00831606102B
:101D5000000086148312861CAB2E0430F700F70BAC
:101D6000AF2EB22E0000831606140430F700F70BD6
:101D7000B72E83125F08F8000800F701F801620827
:101D800003106318F707F70CF80CE318F707F70CC4
:101D9000F80C6319F707F70CF80CE319F707F70CC1
:101DA000F80C631AF707F70CF80CE31AF707F70CAF
:101DB000F80C631BF707F70CF80CE31BF707F70C9D
:101DC000F80C0800DE011F267808DE00DF008A110B
:101DD000ED278A157808C8000130DE001F26780834
:101DE000DE00DF008A11ED278A157808C90002306D
:101DF000DE001F267808DE00DF008A11ED278A1535
:101E00007808CA008A150A16B1288E30F7008316A2
:101E10002108F8002008F900FA01F808031D1A2F1C
:101E20007908F800F9010830F702F808031D1A2FA5
:101E3000F701222F0310F81B212FF90DF80DF703DE
:101E40001A2FF813831208007B080319A32F831697
:101E5000A4002008031D2E2F8312A32FA40703180C
:101E60003C2F7F30A4020318372F8312A32F031DAA
:101E70003B2F8312A32F422F8130A407031C422F34
:101E80008312A32F2408F700F801F901FA017C0856
:101E9000A800A8177D08A7007E08A6001830A40097
:101EA000A501261C6B2F2308FA07031C5D2FF90AD6
:101EB000031D5D2FF80A0319A5172208F907031C53
:101EC000642FF80A0319A5172108FD00FD177D08E6
:101ED000F8070318A517A50DF80CF90CFA0CA80CB7
:101EE000A70CA60C0310A40B502F0130F707031CFE
:101EF0007B2F8312A32FF81B852FA80DFA0DF90D48
:101F0000F80DF70B852F8312A32FA81F982FFA0A1D
:101F1000031D982FF90A031D982FF80A031D982F07
:101F2000F80CF90CFA0CF70A031D982F8312A32F53
:101F30007C08A5002108A506A51FA02FF817A82F2B
:101F4000F813A82F8312F701F801F901FA0183169B
:101F5000831208006308EA006708EA06EA1FB52F43
:101F600003110310E31B0314E82F6308EA0066085B
:101F7000EB006208EB020319C32FEA1FE82F0308E6
:101F8000013A8300E82F6708EB006308EB020319AE
:101F9000CF2FEA1FE82F0308013A8300E82F6808D3
:101FA000EB006408EB020319DB2FEA1FE82F03089C
:101FB000013A8300E82F6908EB006508EB0203197A
:101FC000E72FEA1FE82F0308013A8300E82F0310E8
:101FD00008001030E200F701FA01DF0CDE0C031CF0
:101FE000F72F6008F7070318FA0A6108FA07FA0CD6
:0C1FF000F70CF90CF80CE20BED2F0800C8
:102000008030831C06288316A50683128316AA0136
:10201000AB012108A9002508A90620080319F42806
:10202000A800F70024080319FD28A802031999281D
:10203000031C57282508AE00AE172608AD00270858
:10204000AC00AB010310AE0CAD0CAC0CAB0CA80B90
:102050002128A91F2E282A1411292A1028102A16EF
:10206000A3308400831326292A12A91B4128281C87
:102070004C28AE0CAD0CAC0CAB0CF70A03190C29B8
:102080004C28AE1B4F280310AB0DAC0DAD0DAE0DA3
:10209000F70303190C2941282A17B9282A13210804
:1020A000A900A91F5528AE170529AE130529240834
:1020B000A800F7002008A8022108AE00AE172208E9
:1020C000AD002308AC00AB010310AE0CAD0CAC0CA2
:1020D000AB0CA80B6328A91F7028AA141129AA10F9
:1020E0002810AA16A730840083132629AA12A91B38
:1020F0008328281C8E28AE0CAD0CAC0CAB0CF70A58
:1021000003190C298E28AE1B91280310AB0DAC0DC2
:10211000AD0DAE0DF70303190C298328AA17B928B2
:10212000AA132508A900A91F9728AE170529AE13E1
:1021300005292508AE00AE172608AD002708AC001B
:10214000A91FA628AE132A1511292A11AB012810A0
:10215000A330840083132629A91BCF282108A900B6
:10216000281CB928AE0CAD0CAC0CAB0CF70A03194B
:102170000C29AB1FCA28AC0A031DCA28AD0A031DCF
:10218000CA28AE0A031DCA28AE0CAD0CAC0CF70A67
:1021900003190C292A1B4E28AA1B9028EE288030F0
:1021A000AE06AE1FD72811292508A900E42821086A
:1021B000A900AE08031DE428AD08031DE428AC08FF
:1021C000031DE428F7010529AE1BEE280310AB0D13
:1021D000AC0DAD0DAE0DF70BE4280C29A91FF228AC
:1021E000AE170529AE1305292408F7002508AE000F
:1021F0002608AD002708AC0005292008F7002108B3
:10220000AE002208AD002308AC002E08F8002D080F
:10221000F9002C08FA004429F701F801F901FA0144
:102220004429AB01AC09AD09AE09AB09AB0A031DEA
:102230001F29AC0A031D1F29AD0A0319AE0A2A186B
:102240002D28AA186F282A19A528D4280008AC0719
:10225000031C3029AD0A031D3029AE0A03192814C6
:1022600084030008AD07031C3829AE0A031928149B
:1022700084030008801F803AAE07031828142A1A26
:102280003428AA1A7628AC28831208005E08C300F6
:102290000A12C6230A16F808031DF22ACC30FD00E4
:1022A0000A12FD230A164430FD000A12FD230A1605
:1022B000831686150330FB00FA30FC000A128312E5
:1022C00030220A16FB0B6529672983165C290A123E
:1022D000C6230A160A12C6230A16F8080319732918
:1022E0000030F80092295530FD000A12FD230A162D
:1022F000FB017B08073C031C9029430DF700F70DF9
:10230000F70DF830F70577087B072B3E8400831321
:102310000008FC00FD000A12FD230A16FB0A7929B9
:102320000130F800F8080319EB2ABE30FD000A124C
:10233000FD230A16DF015F08013C031CD32961302D
:102340005F07F800FA010318FA0A7808FB007A0818
:10235000FC00FE01FD017D08073C031CC8290A1290
:1023600021240A16F8080319C1290130F7007D0855
:10237000F8000319BF290310F70DF80BBB297708E4
:10238000FE04F930F700F70BC329C629FD0AAB2973
:102390007E08F8007B08840083137C188317780874
:1023A0008000DF0A9B296208EB006108EA00EB1F4E
:1023B000E9292D30F0006A08FB00FB096B08FC00DE
:1023C000FC0901307B07EA007C08EB000318EB0AEC
:1023D000EB292B30F000EF01EE016A080F39E00025
:1023E0006B0CED006A0CEC00ED0CEC0CED0CEC0C45
:1023F000ED0CEC0C0F30ED05600F032A0130EC07FB
:102400000318ED0A102ADF0160085F020318102A82
:102410009530EE07013003180230EF07DF0A042A77
:1024200070082B3C031D792A6F088316A1008312C4
:102430006E088316A0000A128A15831205270A1651
:102440008A111730FE00B730FD005130FC007130AA
:10245000FB007A088316A3007908A2007808A1007F
:102460007708A0000A128A15831224270A168A11F7
:102470007A08FE007908FD007808FC007708FB0068
:102480006D088316A10083126C088316A0000A123F
:102490008A15831205270A168A1183107A08831673
:1024A000A3007908A2007808A1007708A0007E08A0
:1024B000A7007D08A6007C08A5007B08A400831265
:1024C000002083108316A301A201A101A0017A08B4
:1024D000A7007908A6007808A5007708A400831251
:1024E00000207A08F4007908F3007808F2007708F1
:1024F000F10070082D3C031DE22A6F088316A1002D
:1025000083126E088316A0000A128A15831205270B
:102510000A168A111730FE00B730FD005130FC005A
:102520007130FB007A088316A3007908A2007808AE
:10253000A1007708A0000A128A15831224270A1620
:102540008A117A08FE007908FD007808FC007708F7
:10255000FB006D088316A10083126C088316A0008F
:102560000A128A15831205270A168A1183107A081F
:102570008316A3007908A2007808A1007708A000BC
:102580007E08A7007D08A6007C08A5007B08A400A3
:102590008312002083148316A301A201A101A001CC
:1025A0007A08A7007908A6007808A5007708A40093
:1025B000831200207A08F4007908F3007808F2000A
:1025C0007708F1007108F7007208F8007308F90045
:1025D0007408FA00F22A8930F7000A30F800E03077
:1025E000F900FA018A150A16C8288318FA2AA030B9
:1025F00084008313F701F801F901FA018316A001A1
:10260000A101A201A30176087504740473040319DF
:102610003B2B2030A40003108312EF0DF00DF10DC1
:10262000F20D8316A00DA10DA20DA30D76082302B5
:10263000031D242B75082202031D242B740821027C
:10264000031D242B73082002031C352B7308A002E2
:102650007408031C740FA1027508031C750FA202F5
:102660007608031C760FA3020314F70DF80DF90D7D
:10267000FA0DA40B0B2B20088000840A210880008F
:10268000840A22088000840A23088000831208003C
:102690000408E7006608E90003196D2B6508FE00D1
:1026A0006408FD006308FC006208FB008316A301B8
:1026B000A2012030A1008230A0000A128A158312E4
:1026C00024270A168A117A08E5007908E4007808B8
:1026D000E3007708E200E90B4E2B6508F20064087E
:1026E000F1006308F0006208EF006F08B63CEF00ED
:1026F000FA017008F300F0170310F00CF10CF20C63
:10270000FA0CF90CF80CF70CEF0B7C2BF31F932B46
:10271000F709F809F909FA09F70A0319F80A031978
:10272000F90A0319FA0A7A08E5007908E40078083A
:10273000E3007708E200E51FAA2BE703E716E209AA
:10274000E309E409E509E20A0319E30A0319E40AC3
:102750000319E50A3B30EE009A30ED00CA30EC0078
:10276000EB010A30E90066080319E70A83146230B6
:10277000840083136508F2006408F1006308F00028
:102780006208EF006E08F6006D08F5006C08F400B2
:102790006B08F300F5227808F708031DE22B660AA0
:1027A00069020319E22B67080319E42B0F39690248
:1027B0000319DC2B03181C2CE71B1C2C671BE42BB8
:1027C0002030162C2030E705E71EF42BE7126608B0
:1027D000031DE7037708E7002D30EF000A123D23C1
:1027E0000A166708F700E70166086902031D042C52
:1027F0007708E7002E30EF000A123D230A1667081B
:10280000F7002030E70500303030E71E162CE712C5
:102810006608031DE7037708E7002D30EF000A1272
:102820003D230A166708F700E7013030F7077708FD
:10283000EF000A123D230A1683106E08F2006D089D
:10284000F1006C08F0006B08EF00F601F501F401EF
:102850000A30F300F5227A08EE007908ED007808D6
:10286000EC007708EB00E90BB62B8A110A16682CEE
:102870006108E5006008E4005F08E3005E08E2002C
:10288000E901E8015E30E7008530E6000A128A15AA
:10289000AA270A168A110319702C0130F0000230A1
:1028A000F1000A122B230A160130F4000430F5005F
:1028B0000A12A5220A16023084006108E5006008A9
:1028C000E4005F08E3005E08E2000130E600482B08
:1028D0000130F4000230F5000A12A5220A16802CFD
:1028E0000130F0000230F1000A122B230A165F308B
:1028F00003178D0001308F000A12031361230A169B
:102900008A150A1618290830F0000230F1000A1260
:102910002B230A160130F4000630F5000A12A52216
:102920000A164A08E1000130E2000A121C260A16C3
:102930003A30EF000A123D230A164908E10001303F
:10294000E2000A121C260A163A30EF000A123D2352
:102950000A164808E1000130E2000A121C260A1695
:062960008A150A161B296E
:1030000003081F398300FF30A000A9012A100430F3
:10301000C500C601C701AA10CB01CC0183161F143D
:103020009F141F159F1107309C0083138312D60134
:10303000D501D801D701D9016430FC000A128A11E8
:1030400030220A168A1583161F109F141F119F1114
:103050001F1783121F139F1783169F1783121F14A6
:10306000A0102008831687008312871420112008DF
:10307000831687008312071583160811831208151B
:103080000A128A11E22A0A168A150A128A11122BCA
:103090000A168A150A3003178D0002308F000A12B3
:1030A0008A11031361230A168A150430DE00FA30F0
:1030B000FC000A128A1130220A168A15DE0B5728E4
:1030C0000A128A11CC2C0A168A157808D900D90858
:1030D00003197628143003178D0002308F000A126E
:1030E0008A11031361230A168A15812821300317D8
:1030F0008D0002308F000A128A11031361230A1611
:103100008A150430DE00FA30FC000A128A113022DF
:103110000A168A15DE0B83280C30EF000A128A117A
:103120003D230A168A150A128A1105250A168A15E0
:103130007808C600C6080319AF2883160811831241
:1031400008150A1200280A160830DE00FA30FC00C2
:103150000A128A1130220A168A15DE0BA6280A12D4
:10316000E22E0A163230FC000A128A1130220A16A8
:103170008A15D9080319D8280130F000F1000A1285
:103180008A112B230A168A150130DE008A1146297E
:103190008A157A08D0007908CF007808CE00770821
:1031A000CD003230FC000A128A1130220A168A152C
:1031B00003178D0183168C130C1483120C088316CD
:1031C0000313A101A0000A12831205270A167A0828
:1031D000D4007908D3007808D2007708D1005408C9
:1031E000E5005308E4005208E3005108E200E90159
:1031F000E8017F30E7008630E6000A12AA270A16A7
:10320000031D0829D401D3014830D2008330D100F6
:10321000C708031D872BD908031919295008E10095
:103220004F08E0004E08DF004D08DE008A11382C00
:103230008A158A11832C8A15D90803195029E501AA
:10324000E4016830E3008330E2005008E9004F08F1
:10325000E8004E08E7004D08E6000A12AA270A1601
:1032600003183429031D5029C808031D5029F430C0
:10327000DE000A128A117C250A168A150530F00034
:103280000130F1000A128A112B230A168A15013027
:10329000F4000330F5000A128A11A5220A168A15D5
:1032A0004A08113C031C58294A08073C031C5D29A5
:1032B00083160811831208156129831608118312D9
:1032C00008115008E5004F08E4004E08E3004D08DF
:1032D000E200E901E030E8000A30E7008930E6006A
:1032E0000A12AA270A160319D229D9080319D229C2
:1032F0005008E5004F08E4004E08E3004D08E200E6
:103300005408E9005308E8005208E7005108E600B5
:103310000A12AA270A16031CA3290130F000F100A3
:103320000A128A112B230A168A150130F400F500BF
:103330000A128A11A5220A168A152011200883165E
:103340008700831207155408E5005308E40052086B
:10335000E3005108E2005008E9004F08E8004E0879
:10336000E7004D08E6000A12AA270A16031CD12915
:103370000130F000F1000A128A112B230A168A1577
:103380002B3003178D0002308F000A128A110313AD
:1033900061230A168A1520112008831687008312DC
:1033A0000711EB290130F000F1000A128A112B23DA
:1033B0000A168A152C3003178D0002308F000A126E
:1033C0008A11031361230A168A1520112008831617
:1033D000870083120711013003178D0083168C13A9
:1033E0000C1483120C0803134A02031C1A2A02301D
:1033F00003178D0083168C130C1483120C0803130F
:103400004902031C1A2A0230F0000130F1000A12AE
:103410008A112B230A168A150130F400F5010A12CD
:103420008A11A5220A168A15A01020088316870083
:1034300083128714033003178D0083168C130C142A
:1034400083120C0803134A02031C4C2A043003178E
:103450008D0083168C130C1483120C08031349027D
:10346000031C4C2A0230F0000130F1000A128A11CC
:103470002B230A168A152D3003178D0002308F007A
:103480000A128A11031361230A168A15A010200854
:103490008316870083128710053003178D0083166B
:1034A0008C130C1483120C080319012B05308D00AA
:1034B00083168C130C1483120C080313DE004C08C3
:1034C0004A025E020319662A0318002B0330F0003B
:1034D0000130F1000A128A112B230A168A150130D5
:1034E000F4000530F5000A128A11A5220A168A1581
:1034F000A01120088316870083128715D708031DA3
:10350000A52AD808031DA52ADF014A08DE000E30CF
:10351000E1001030E0000A12E9270A167908DF00FE
:103520007808DE004908E2003C30E3000A12BD26BC
:103530000A167808DE070318DF0A48085E07D70076
:103540005F08D8000318D80A002BDF014A08DE0004
:103550000E30E1001030E0000A12E9270A1679085F
:10356000DF007808DE004908E2003C30E3000A1280
:10357000BD260A167808DE070318DF0A4808DE07AA
:103580000318DF0A57085E02DA005F08DB005808FC
:10359000031C580FDB020530F0000130F1000A1265
:1035A0008A112B230A168A15063003178D008316FD
:1035B0008C130C1483120C0803135A020319002BEA
:1035C000031C002BA011200883168700831287118B
:1035D000D801D7014A08CC000330F0000130F100D7
:1035E0000A128A112B230A168A152E3003178D0012
:1035F00002308F000A128A11031361230A168A15FA
:10360000031707308D0083168C130C1483120C08DB
:103610000319882B07308D0083168C130C1483122A
:103620000C080313DE004B084A025E0203191A2B32
:103630000318872B0430F0000130F1000A128A11C0
:103640002B230A168A150130F4000730F5000A1200
:103650008A11A5220A168A158316081083120814E7
:10366000D508031D422BD608031D422B4A08E20051
:103670003C30E3000A12BD260A1649087807D50037
:10368000D601872B4A08E2003C30E3000A12BD262F
:103690000A1649087807F80055087802DC00DD01B1
:1036A0005608031C560FDD020530F0000130F10012
:1036B0000A128A112B230A168A15083003178D0067
:1036C00083168C130C1483120C0803135C02031969
:1036D000872B031C872B8316081083120810D60132
:1036E000D5014A08CB000430F0000130F1000A1285
:1036F0008A112B230A168A152F3003178D000230EA
:103700008F000A128A11031361230A168A15031700
:063710000313932863007F
:0200000401E019
:090000001A0801120200000000C0
:020000040000FA
:02400E00323F3F
:00000001FF
